:020000020000FC
:100000000CC118E01A95F1F708950AE0409508949C
:1000100010F4599A02C059980000F3DFF2DF4695B8
:100020000A95B1F708951FEF2AE02A95F1F71A957E
:10003000D9F70895A52F12D05A2F08950FD00895FB
:100040002A9A229A2D98259A2B98239A24980895D3
:100050002D982B982A9808952A9A089518E0550FFC
:1000600010F42B9A02C02B9800002D9A1058105EA5
:10007000F0F32D981058105EF0F31C9953951A95D3
:1000800071F708952A9857EDD5DFD8DF57FFFDCFD8
:100090002A9A089560E070E080E090E05D982A98E8
:1000A00052E8C8DF262F372F220F331F532FC2DF0E
:1000B000522FC0DF50E0BEDF51E0BCDFBBDFBADF54
:1000C000B9DF562FB7DF572FB5DF16E020E0810FDD
:1000D000921F562FAFDF462F98DF472F96DF482F0E
:1000E00094DF492F92DF452F90DF11E020E0810F50
:1000F000921F883011E0910760F32A9A11E020E006
:10010000610F721F603012E0710708F008F4C4CF6D
:100110005D9A0895459860E070E02A9852ED8ADF74
:10012000262F372F220F331F532F84DF522F82DFCA
:1001300050E080DF50E07EDF7DDF7CDF7BDF80E032
:1001400090E07CDF462F61DF472F5FDF482F5DDFC8
:10015000492F5BDF452F59DF11E020E0810F921F0F
:10016000883011E0910768F32A9A11E020E0610FCE
:10017000721F603012E0710710F060E070E04F9B7A
:10018000CCCF2A9A459A0895459860E070E080E0C7
:1001900090E02A9858EE4EDF262F372F220F331F7C
:1001A000532F48DF522F46DF50E044DF50E042DF5C
:1001B00041DF40DF3FDF42DF462F27DF472F25DFCC
:1001C000482F23DF492F21DF452F1FDF4F9BF3CF20
:1001D0002A9A459A089560E070E0862F972F880F3D
:1001E000991F492F12DF482F10DF11E020E0610F27
:1001F000721F603012E0710780F3089560E070E0D4
:10020000462F03DF472F01DF11E020E0610F721F4F
:10021000603012E07107A0F3089510E820E0109319
:1002200061002093610014E01EBF1FEF1DBF519AB3
:10023000599A3D9A459A559A5D9A56985E9A57985A
:0E0240005F9AFEDE4E9B26DF4F9B9EDFFBCFBC
:00000001FF
